:1000000000308A00AC2900000A108A100A11820709
:10001000003400340634403420340134FF343F349B
:10002000ED3409342D341234DB34243400340134FB
:100030003134003407340034C0343F34C034093420
:1000400000341034C03400340034403400341234EE
:100050003F34123400340934DB3400348F3400343C
:10006000E634003469340434FD340034013412348D
:10007000FF340034E734003400341C3400342334BB
:1000800000340634C834003400343034A334083427
:10009000BB340134F7340034BF3400343934003415
:1000A000DE3400347934003471340034BD3400342B
:1000B000F6340034093409341E3400347034063404
:1000C0003834003436342234363424343F34003467
:1000D000F33400343F340434F3340434ED34003466
:1000E000013409343E34003430341234363414349C
:1000F0000034363400342A34093412346034003485
:10010000003424348234003400342234083400347F
:1001100000342034F7340034BF3400343934003430
:10012000DE3400347934003471340034BD340034AA
:10013000F6340034093409341E3400347034063483
:100140003834003436342234363424343F340034E6
:10015000F33400343F340434F3340434ED340034E5
:10016000013409343E34003430341234363414341B
:100170000034363400342A3409341234403406341E
:100180000034093480343034C03412340A108A10F8
:100190000A11820747346F34743420347634613462
:1001A0006C343A3420343034783425344C34583478
:1001B0000A340D3400340A108A100A1182075234AE
:1001C0006534613464347934203474346F342034C9
:1001D00064346934733470346C34613479342E345B
:1001E0000A340D340034A0132008831687008312CC
:1001F00087130830F800000000000000F8170F29EE
:10020000F813A80C03188717031C871378170F29F6
:100210007813F80B01290000000000008717A730B1
:100220008400840B11290000F81B0029781B082981
:1002300000340830F7002017200883168700831247
:10024000071B2029A401F7173329F71333290310BB
:10025000071B0314A40C771733297713F70B2729EF
:100260002408F8003F29A730F71B2D30F800F80BC1
:1002700037290000F71B2529771B2D2927298A11EB
:100280000A12CE29A71B54290F30F700260EF705B6
:100290000A30770203184F293030F7075129270811
:1002A000F7077708A800F3200F30A6050A302602CA
:1002B00003185C2930305E29A7132708A6072608F3
:1002C000A800F32000342408A50025081F3C0318CB
:1002D0007D2925087E3C031C7D292030A5020310C2
:1002E000250DF700A600260A0420FA00260804209F
:1002F000F8007A08F900802980290030F800F90018
:100300007908A3007808A200A5012508C620A50A3F
:10031000A800F3200B302502031D85292308A60021
:100320003730A70042212208A6003730A70042211B
:100330000A30A800F3200D30A800F3202308A600FF
:100340002208A5002508FF3A8600A8012608FF3AE2
:1003500088008A110A12F62984011F3083050730AC
:1003600083169F00FF308312A000A013200883167D
:100370008700831287178316091286018801FF30D0
:10038000831286008800A4012408DB20A40AA800A8
:10039000F32013302402031DC42919297808A10071
:1003A00021088400003000040319DF290408A40098
:1003B0000008A800F32024088400840AD2292030F1
:1003C000A800F3203D30A800F3202030A800F3203F
:1003D0002108A6003730A70042210A30A800F320E8
:1003E0000D30A800F3202108A4006329CD29630063
:02400E007A3FF7
:00000001FF
